:020000040000FA
:06000000B3EF0FF0120047
:06080000B3EF0FF012003F
:0608080032EF0CF01200BB
:0608180032EF0CF01200AB
:06082A000200CC1F0000DB
:10083000000200000B000000CA1F000015020000AB
:0408400002000000B2
:0C0844005EEC09F0FB0EDBCFF3FFDB06DF
:10085000F35000090AE0ACEC09F0FA0E17EC0AF0CC
:10086000F3E1151CF1E1010E01D0000E8DEF09F04E
:100870005EEC09F03B0EE12402E3E168E652E16E32
:10088000010EDB6A020EDB6AF90EDBCFF6FFFA0E11
:10089000DBCFF7FFFB0EDBCFF8FF0800F550DF6E74
:1008A000DF5002E1B1EF08F0250EDF5C02E0A4EFBB
:1008B00008F0030EDB6A040EDB6A050EDB6A060E27
:1008C000DB6A070EDB6AC6EC08F02D0EDF5C0CE07D
:1008D0002B0EDF5C09E0200EDF5C06E0230EDF5C00
:1008E00003E0300EDF5C1AE1DF50300A14E0130A37
:1008F0000FE0030A0AE00B0A05E0060AE4E1030E32
:10090000DB80E1D7030EDB82DED7030EDB84DBD78F
:10091000030EDB86D8D7030EDB88D5D72A0EDF5C23
:100920001BE1C2EC08F010EC09F010E0030EDB80D4
:1009300008680968130EDBCF0DF0140EDBCF0EF044
:10094000A8EC0EF0040E06C0DBFF03D0130EF9EC8A
:1009500008F0C6EC08F00BD0090EDB6A67EC09F072
:1009600003E0DBEC09F0FAD7090EF9EC08F0030E0E
:10097000DBB0DB982E0EDF5C1BE1C6EC08F02A0E24
:10098000DF5C0BE1C2EC08F010EC09F003E1130EA0
:100990004BEC09F0C6EC08F00BD0090EDB6A67ECF3
:1009A00009F003E0DBEC09F0FAD7090E4BEC09F093
:1009B000680EDF5C07E1C6EC08F0680EDF5C1DE145
:1009C000030E18D0740EDF5C17E07A0EDF5C14E0C3
:1009D000480EDF5C06E0540EDF5C03E05A0EDF5C7D
:1009E00002E1020E07D06C0EDF5C03E06A0EDF5CF2
:1009F00004E1010E9EEC09F0C9DBDF506E0A01E153
:100A00007FD31E0A01E192D1200A01E18FD13F0A72
:100A100001E149D11A0A01E146D10D0A01E143D1B0
:100A2000200A01E140D13A0A01E13DD1200A01E169
:100A30003AD1260A01E135D10D0A01E132D11A0A73
:100A400001E1D9D0200A4AE0300A1FE0460A0EE050
:100A5000250A01E083D3D950F90FE96EFF0EDA20A1
:100A6000EA6E010EEE5E000EEE5AEE5AACEC09F0A4
:100A7000250EE66E95DB03E1151C01E169D3A8ECB8
:100A800009F001E26BD3DB2A69D3080EDB6A040E9E
:100A9000DB50010806E2040EDB0470EC09F0DB50C9
:100AA0008BDB080EDB5009E0030EDB50010B05E188
:100AB00072DB01E04DD3080EDB6A64DBEFCFDFFFB2
:100AC00020EC0AF003E1151C01E142D3A8EC09F087
:100AD00001E3DB2A60DB01E141D33AD3070EDB50AF
:100AE00002080FE1ECEC09F0030EB3EC09F00E0E76
:100AF000EECFDBFF0F0EEECFDBFF100EEECFDBFFF6
:100B000020D0F70EDBCF17F0F80EDBCF18F0020E77
:100B1000175E000E185AF70E17C0DBFFF80E18C04C
:100B2000DBFF17C0E9FF18C0EAFFA3EC09F0166A63
:100B30000E0E14C0DBFF0F0E15C0DBFF100E16C02B
:100B4000DBFF0E0EDBCFE6FF0F0EDBCFE6FF100E56
:100B5000DBCFE6FF83EC0EF0E552E552E552130ED3
:100B600007C0DBFF140E08C0DBFF060EDB5005E0FC
:100B7000130EE7EC09F001E26ADB0BEC0AF002E28B
:100B8000130E37DBCEEC09F006E0040EE7EC09F0BB
:100B900002E2050E2EDB030EDBB005D0FCDA01E02D
:100BA000D7D2080EDB6A090EDB6A0E0EDBCFF6FF2A
:100BB0000F0EDBCFF7FF100EDBCFF8FF0800F5506C
:100BC000DF6EDF5014E011EC0AF011E220EC0AF0C5
:100BD00003E1151C01E1BCD2BBDB01E3DB2A090EFA
:100BE000DB2AD9500E0FE96E000ECBDBE7D7D3DA44
:100BF00001E1B4D2ADD2C6DA110EEECFDBFF120E98
:100C0000EDCFDBFF110EDBCFE6FF120EDBCFE6FFF1
:100C100075EC0EF0E552E552130EF3CFDBFF140E28
:100C2000F4CFDBFF060EDB5004E0130ED0DB01E255
:100C30000EDB0BEC0AF002E2130EDBDAAFDB05E0B1
:100C4000040EC5DB02E2050ED4DA030EDBB005D0DC
:100C5000A2DA01E07DD2080EDB6A090EDB6A110E12
:100C6000DBCFE9FF120EDBCFEAFFEFCFDFFFDF5074
:100C700014E0D7DB12E2E4DB03E1151C01E168D2EA
:100C800067DB01E3DB2A090EDB2A110EDB2ADBCF4F
:100C9000E9FF120EE8E3DB2AE6D77DDA01E15ED256
:100CA00057D2030EDB8E070EDB0410E195DB040E3A
:100CB0005ADB0A0EEECFDBFF0B0EEECFDBFF0C0E86
:100CC000EECFDBFF0D0EEECFDBFF6CD0070EDB505F
:100CD00003082CE1030EDBAE0DD0B2DA020E76DA99
:100CE000EFCF14F0156A166A176A14AE39D015687A
:100CF000166835D0F70EDBCF15F0F80EDBCF16F007
:100D0000020E155E000E165AF70E15C0DBFFF80E28
:100D100016C0DBFF15C0E9FF16C0EAFFEFCF14F0E5
:100D20000A0E14C0DBFF0B0EDB6A38D0070EDB5057
:100D3000020809E1030EDBAE04D059DB16AE10D079
:100D40000ED055DB0DD0030EDBAE12D079DA020ED9
:100D50003DDAF9DA166A176A15AE02D01668176816
:100D6000E2DA0C0E16C0DBFF0D0E17C0DBFF1AD047
:100D7000F70EDBCF16F0F80EDBCF17F0020E165E83
:100D8000000E175AF70E16C0DBFFF80E17C0DBFF78
:100D900016C0E9FF17C0EAFFD6DAC5DA0C0EDB6A27
:100DA0000D0EDB6A060EDB5005E1010EF36E050E3B
:100DB000F3CFDBFF150EDB6A160EDB6AD950370F57
:100DC000146E000EDA20156E390E14C0DBFF3A0ED9
:100DD00015C0DBFF380EDB6A080EDB6A0A0EAEDADE
:100DE000DF50780A12E0200A10E0280A0CE0200AFE
:100DF0000AE03F0A06E00D0A02E0200A08E1020EBE
:100E000005D0080E03D0080EDF26100E97DA030E69
:100E1000DBBE02D0DB92DB94DB50800B24E08ADA6D
:100E2000D890030EEB50000A08E6000EEE5C000EB0
:100E3000EE58000EEE58000EEE5815E213DA0B686D
:100E40000C680D680E683DEC0EF00A0E02C0DBFF68
:100E50000B0E03C0DBFF0C0E04C0DBFF0D0E05C044
:100E6000DBFF2D0E08D0030EDBA202D02B0E03D029
:100E7000DBA408D0200EF36E170EF3CFDBFF150EA8
:100E8000DB2A02D0170EDB6A050EDB5003E1B7D96F
:100E900001E189D0B40E146E1F0E156E000E166E91
:100EA000070EDBCF17F0186A196A1A6A17C00BF021
:100EB00018C00CF019C00DF01AC00EF0D3D9FCEC1C
:100EC0000EF014500224F36E15500320F46E1650E9
:100ED0000420F86EF4CFF7FFF3CFF6FF0800090EF9
:100EE000F5CFDBFF580EDF5C0FE1610EF36E090EEC
:100EF0007BD90AE3200E146E090EDBCFE7FF1450F6
:100F0000E75E090EE7CFDBFF070EDBCF14F0156AB3
:100F1000166A176A0FDA14C00BF015C00CF016C071
:100F20000DF017C00EF0EECF06F0EECF07F0EECFCB
:100F300008F0EFCF09F0FCEC0EF009C0EDFF08C09F
:100F4000EDFF07C0EDFF06C0EFFF390EDBCFE9FF75
:100F5000DB063A0EDBCFEAFF01E2DB06090EDBCF50
:100F6000EFFF150EDB2A4BD995E1030EDBA61DD052
:100F70006F0EDF5C06E1C1D918E3150EDB285BDAE2
:100F800014D0780EDF5C09E0580EDF5C06E0620EDC
:100F9000DF5C03E0420EDF5C08E1020EF36E160E2A
:100FA000F3CFDBFF02D0150EDB6A030EDB50100B14
:100FB0000EE0040EDBCF14F0050EDB50D880145485
:100FC00006E2060EDB5003E1040EDB5034DA95D95D
:100FD0000AE2050EDBCFE7FF150EDB50E75E050EDC
:100FE000E7CFDBFF02D0050EDB6A040EDBCF14F087
:100FF000160E45D9D880145414E2160EDBCFE6FF46
:10100000150EDBCFE6FF040EDBCFE6FF050EDB504F
:10101000E552E75CE552D880E754E552D880E754C2
:101020005FD9030EDB50010B0BE1080EDB5008E02B
:10103000B2D801E08DD0080EDB50BED8080EDB6AB6
:10104000170EDB5007E088D9170EF1D903E1151C04
:1010500001E17ED0160EDB5016E07ED9300EE66E32
:101060009FD802E1151C74E077D9DFCFE6FFFBECD7
:101070000DF0E552E552E552F4CF15F00001F31CF6
:1010800002E1151C65E0050EDBCF14F0160EDB50F7
:10109000D880145409E2050EDBCFE7FF160EDB50B3
:1010A000E75E050EE7CFDBFF300EE66E050ECBD90F
:1010B0004FE1390EDB2ADBCFE9FF3A0E01E3DB2AF1
:1010C000DBCFEAFF090EEFCFDBFFDB500EE044D9A8
:1010D000090EADD902E1151C3BE0390EDB2ADBCF4E
:1010E000E9FF3A0EEDE3DB2AEBD755D831E1160ED6
:1010F000DBCFE6FF080EC3D8E552E7245DD82ED03B
:10110000070EDB50030A1CE0010A14E0030A07E0A3
:101110007BD9DBCFEEFF020EDBCFEDFF1FD0F5D882
:10112000196A17AE02D0186819682CD8BCD819C033
:10113000EEFF14D0EAD817BE186824D8B4D80ED061
:1011400063D9DBCFEFFF0AD07BD905E1151C03E1A2
:10115000F368F46810D0FCD801E3DB2A79D94DEFAD
:1011600004F0010EDBCF14F0020EDBCF15F014C03B
:10117000F3FF15C0F4FF3B0EE15C02E2E16AE552C9
:10118000E16ECBD029D9020EB3EF09F061D9080086
:10119000F550DF6E1200200EE66E080E23EF0AF007
:1011A000FBEC0DF0E552E552E552F3CF14F0F4CF2D
:1011B00015F00001F31C1200146E156AD950010FCE
:1011C0004DD91450EE261550ED221200185E000E77
:1011D000195AF70E18C0DBFFF80E19C0DBFF18C054
:1011E000E9FF19C0EAFF1200DBCFF4FFF350F45C13
:1011F0001200DB50E76E040EE7CFDBFF12000A0E91
:10120000DBCF14F00B0EDBCF15F00C0EDBCF16F09E
:101210000D0EDBCF17F0145015101610171012001A
:10122000130EEECFDBFF140EEDCFDBFF130EDBCF83
:1012300014F0140EDBCF15F00001800E151412000F
:10124000F70EDBCF18F0F80EDBCF19F01200050E09
:10125000DB50E66ED950130F01D9E552E750EE6E20
:10126000ED6A12000A0EDBCF06F00B0EDBCF07F0A3
:101270000C0EDBCF08F00D0EDBCF09F01200DBCF38
:10128000E6FF150EDBCFE6FF050EDB50E552E72447
:10129000E552E7241200DB50CED8010EF36E060EA5
:1012A000F3CFDBFF1200EE50EFCFEAFFE96E16C07E
:1012B000EEFF17C0EEFF18C0EEFF1200D9CFE6FF19
:1012C000DACFE6FFE1CFD9FFE2CFDAFF1200DFCFBE
:1012D000E6FFE66A91EC0FF0E552E552F35012009A
:1012E000E76E080EE7CFDBFF1200EECF14F0EECF73
:1012F00015F0EFCF16F0176A1200050EDBCF14F0D1
:10130000150EDB50D88014541200010EDBCF16F0FE
:10131000020EDBCF17F0186A1200E552E5CFDAFFB4
:10132000E7CFD9FF12000A0E14C0DBFF0B0E15C069
:10133000DBFF1200D9500A0F2EEF0AF0F36E070EF2
:10134000F3CFDBFF1200EECF14F0EFCF15F0120059
:10135000010EDB2A020E1200FC0EDBCFE6FFFD0EB3
:10136000DBCFE6FF1200145E000E155AF70E14C014
:10137000DBFFF80E15C0DBFF14C0E9FF15C0EAFF64
:101380001200DA20EA6EEF2AEECFF6FF000EEF220F
:10139000EECFF7FFEF22EECFF8FF1200040EDBCF07
:1013A000E6FF130EDB50E552E75C9ADFDB5004DF0B
:1013B000060EDB501200090EDB500A0DF350DF243D
:1013C000D00FE76E090EE7CFDBFFC6EF08F0DB506A
:1013D000F36E050EF4EF08F0F70EDBCF14F0F80E05
:1013E000DBCF15F01200DFCFE6FFD0EF08F028DFEB
:1013F000030EECDE75EF09F022EC04F0E552E55245
:10140000E552E55200091200BDDEEE50EFCFEAFFD3
:10141000E96E010E1200130EDB50F36E040EF4EFB2
:1014200008F0040EDB50F36E090EF4EF08F0DBCF8A
:10143000E6FFD0EF08F0E76E050EE7CFDBFF120006
:101440008BDFF3EF09F0DBCFE6FF86DFFCEF09F07F
:10145000D950F90FE96EFF0EC1EF09F0E96E000EE9
:06146000DA20EA6E120022
:0A1466004D0EE66EE66A6C0EE66EAF
:10147000B6EC0DF0E552E552E5521200D9CFE6FF89
:10148000E1CFD9FF040EE126DE6ADE6ADE6ADD6A9C
:10149000DD52DD52D9CFE9FFDACFEAFFD890030E53
:1014A000EB50000A08E6400EEE5C0D0EEE58030EFF
:1014B000EE58000EEE5811E29EAA04D020EC0FF078
:1014C0000ED001D000D0D9CFE9FFDACFEAFFEE2A63
:1014D000000EEE22EE22EE22DDD7000E00D0146EBA
:1014E000040EE15C02E2E16AE552E16E1450E5525D
:1014F000E7CFD9FF1200D9CFE6FFE1CFD9FFE652FF
:101500009EAAFED720EC0FF0DF6EDF5000D0E55230
:10151000E552E7CFD9FF1200D9CFE6FFE1CFD9FFDF
:10152000E6529EAAFED720EC0FF0DF6EDFCFE6FF7B
:101530007AEC0FF0E552DF5000D0E552E552E7CFEC
:10154000D9FF1200D9CFE6FFE1CFD9FFE65203C29F
:10155000DFFF0201036BDF5000D0E552E552E7CF19
:10156000D9FF120000C2F3FF01C2F4FF00D0120045
:10157000D9CFE6FFE1CFD9FFE6523FEC0FF0F350B1
:10158000DF6EF29E02010251146E156AD89015505A
:1015900004E68D0E145C000E155805E20201185188
:1015A000DF5C02010227F28EDFCF18F2E552E5522E
:1015B000E7CFD9FF1200D9CFE6FFE1CFD9FF030E65
:1015C000E126DF6A8150100B01E0010EE76E010E8B
:1015D000E7CFDBFF3FEC0FF0F3500201D88004555A
:1015E000E76E020EE7CFDBFF3FEC0FF0F3CF04F224
:1015F00002010251146E156AD890155004E68D0E42
:10160000145C000E155802E3010E086F026B0851BE
:101610000CE00A5109E0010EDB5006E1086B096B92
:101620000D0E056F066B076BE7D00A516EE1010ED8
:10163000DB506BE0095125E1020EDB50146E156A98
:10164000200E145C000E15581CE3020EDB50166EC3
:10165000176A330ED8801654000E175412E3055142
:10166000CFEC0FF0F35002010613F45007130551AD
:10167000000802E2050702D0010EDF6E010E096FBD
:1016800044D0095125E1020EDB50146E156A400E5C
:10169000145C000E15581CE3020EDB50166E176A20
:1016A000660ED8801654000E175412E30551CFEC85
:1016B0000FF0F35002010613F45007130551000810
:1016C00001E20507055102E1010EDF6E096B1DD035
:1016D000090519E1020EDB50146E156A200E145C28
:1016E000000E155810E3020EDB50166E176A330E0B
:1016F000D8801654000E175406E3096B055102E119
:10170000010EDF6E02D0010E086F0A5175E0010E66
:10171000DB5072E109512BE1020EDB50146E156AA9
:10172000200E145C000E155822E3020EDB50166EDC
:10173000176A330ED8801654000E175418E305515B
:10174000CFEC0FF0F3CF14F0F4CF15F0141E151EEC
:10175000145002010617155007170551000802E240
:10176000050702D0010EDF6E010E096F45D0095149
:101770002AE1020EDB50146E156A400E145C000E56
:10178000155821E3020EDB50166E176A660ED880DC
:101790001654000E175417E30551CFEC0FF0F3CF9A
:1017A00014F0F4CF15F0141E151E14500201061784
:1017B000155007170551000802E2050702D0010E77
:1017C000DF6E096B19D0090515E1020EDB50146EAE
:1017D000156A200E145C000E15580CE3020EDB5047
:1017E000166E176A330ED8801654000E175402E393
:1017F000096B02D0010E086F010EDBCF0AF20C0E4E
:10180000055D08E10739156AE830070B146E1450BE
:10181000010B0AE00B0E055D09E10739176A0F0B92
:10182000166E1650010B02E1010E086F055110E112
:10183000DF500EE00651001902E10751011906E0E0
:1018400006C200F207C201F2010E036F010E086F1B
:10185000030EE15C02E2E16AE552E16EE552E7CF98
:10186000D9FF1200D8CFE4FFE0CFE4FFE46EDACF77
:10187000E4FFE2CFDAFFE9CFE4FFEACFE4FFF6CFFF
:10188000E4FFF7CFE4FFF5CFE4FFF3CFE4FFF4CFBD
:10189000E4FFFACFE4FF00EE00F0140EE80403E3E7
:1018A000EECFE4FFFBD700EE14F00C0EE80403E3E8
:1018B000EECFE4FFFBD7E652F2A006D093908A80E9
:1018C0007ADE93908A90F290E55200EE1FF00C0EB3
:1018D000E80403E3E5CFEDFFFBD700EE13F0140EB1
:1018E000E80403E3E5CFEDFFFBD7E5CFFAFFE5CF53
:1018F000F4FFE5CFF3FFE5CFF5FFE5CFF7FFE5CF49
:10190000F6FFE5CFEAFFE5CFE9FFE5CFDAFFE550E7
:10191000E5CFE0FFE5CFD8FF1000D9CFE6FFE1CF5C
:10192000D9FF030EE126BF0E946E9388570EE66E24
:101930005EEC0FF0E55297DDF2868150100B01E06E
:10194000010EE76E020EE7CFDBFFF290F28E93906E
:101950008A80E00E146E1D0E156E166A14C0E6FF26
:1019600015C0E6FF16C0E6FF6AEC0DF0E552E55241
:10197000E55293908A90E6DD000951E0F3DDF3CF64
:10198000DEFFF4CFDDFFDECF14F0DDCF15F03F0E2C
:101990001416000E151614C0E6FF15C0E6FFDECFC4
:1019A00018F0DDCF19F01950196AE830E830E83046
:1019B0001F0B186E1850010B02E1000E01D0010E32
:1019C000166E176A16BE176816C0E6FF17C0E6FF48
:1019D000DECF1AF0DDCF1BF0060ED8901B321A3284
:1019E000E804FBE11F0E1A16000E1B161AC0E6FFD4
:1019F0001BC0E6FFDECFE6FFDDCFE6FFAA0E1C6EC2
:101A00001D0E1D6E1E6A1CC0E6FF1DC0E6FF1EC037
:101A1000E6FF6AEC0DF01F6E0B0EE15E1F50A8DDB5
:101A2000AAD7030EE15C02E2E16AE552E16EE552FB
:061A3000E7CFD9FF120010
:0A1A36002A0EF66E080EF76E000E81
:101A4000F86E02010900F550106F0900F550116F92
:101A500003E1106701D03DD00900F5500B6F09007C
:101A6000F5500C6F0900F5500D6F09000900F55095
:101A7000E96E0900F550EA6E090009000900F55009
:101A80000E6F0900F5500F6F09000900F6CF12F232
:101A9000F7CF13F2F8CF14F20BC2F6FF0CC2F7FF28
:101AA0000DC2F8FF02010E5302E10F5307E00900D7
:101AB000F550EE6E0E07F8E20F07F9D712C2F6FFE7
:101AC00013C2F7FF14C2F8FF02011007000E115BEA
:041AD000BFD712006A
:0C1AD400D9CFE6FFDACFE6FFE1CFD9FF63
:101AE000E2CFDAFFE652E652E652E652D950FB0F59
:101AF000146EFF0EDA20156E14C0DEFFDD6EDECF31
:101B0000E6FFDDCFE6FFFB0EDBCFE6FFFC0EDBCF13
:101B1000E6FFFD0EDBCFE6FF15C2E6FF16C2E6FFCD
:101B200038EC04F0146E070EE15C02E2E16AE55263
:101B3000E16E1450020EF3CFDBFF030EF4CFDBFF98
:101B4000020EDBCF14F0030EDBCF15F014C0F3FF51
:101B500015C0F4FF040EE15C02E2E16AE552E16EB9
:0C1B6000E552E5CFDAFFE7CFD9FF120015
:041B6C00D9CFE6FFE8
:101B7000DACFE6FFE1CFD9FFE2CFDAFFAC6AAB6A9A
:101B8000FD0EDBB0AC88DBA202D0AC8CAB8CDBB43E
:101B9000AC8EDBA602D0AB8801D0AB8ADBB8AC84BC
:101BA0009E98DBBAAB86DBAC02D09D8A01D09D9AB1
:101BB0009E9ADBAE02D09D8801D09D98FB0EDB5033
:101BC000AF6EFB0EFC0EDBCF15F015C014F0156ADE
:101BD0001450B06EAC8AAB8E949C948EAC50100BAB
:101BE00004E0AC50800B01E1948CE552E5CFDAFFC4
:061BF000E7CFD9FF12004F
:0A1BF600D9CFE6FFDACFE6FFE1CF1A
:101C0000D9FFE2CFDAFFFB0EDBCF14F0FC0EDBCF07
:101C100015F00001800E15141AE1FB0EDBCFE9FF71
:101C2000FC0EDBCFEAFFEECFF3FFEDCFF4FFEE2AA1
:101C3000000EEF22F3CFE9FFF4CFEAFFFD0EDBCF7A
:101C4000EFFFEF50156AF36E15C0F4FF10D0FB0ED6
:101C5000DB50FE0806E1FD0EDBCFE6FFC1EC0FF026
:101C600005D0FD0EDBCFE6FFE3EC0FF0E552E552C9
:0A1C7000E5CFDAFFE7CFD9FF12003D
:061C7A0006500B02F3CF3F
:101C800002F0F4CF03F00C02F3500326000EF42010
:101C9000046E06500D02F3500426000EF420056E6B
:101CA00006500E02F350052607500B02F350032690
:101CB000F4500422000E052207500C02F3500426B3
:101CC000F450052207500D02F350052608500B0270
:101CD000F3500426F450052208500C02F350052658
:0A1CE00009500B02F3500526120014
:061CEA00FE0EE3CFE9FF4E
:101CF000FF0EE3CFEAFFF36AF46AEE5203E0F34A21
:101D0000F42AFBD71200FF0EE3CFF8FFE552FF0ED7
:101D1000E3CFF7FFE552FF0EE3CFF6FFE552E66AA9
:101D2000E66AE66A0900F55209E0FD0EE32A05E1DC
:101D3000FE0EE32A02E1FF0EE32AF4D7FD0EE3CF05
:101D400007F0FE0EE3CF08F0FF0EE3CF09F012001C
:101D500009C013F008C012F008500D02F4CF07F0CC
:101D6000F3CF06F009500E02F4CF09F0F3CF08F0DC
:101D70000D02F3500726F4500822E86A0922125097
:101D80000E02F3500726F4500822E86A09220EAE2C
:101D9000CEEF0EF01250085E1350095A13AE000C2D
:0A1DA0000D50085E0E50095A000CA9
:061DAA0052433520436F97
:101DB00064653D307825303458204465764164644C
:101DC000723D30782530325820546F67676C653D1E
:101DD000256420436D643D3078253032580A0D006B
:101DE0002A2A2A20433138205243352044656D6F1A
:081DF00021202A2A2A0A0D0015
:081DF800056A046A036A026A2D
:101E0000200EE76ED89006360736083609360236B9
:101E10000336043605360B50025C0C5003580D5047
:101E200004580E50055809E30B50025E0C50035A3B
:101E30000D50045A0E50055A062AE72EE4D7120018
:101E4000D9CFE6FFDACFE6FFE1CFD9FFE2CFDAFF65
:101E5000E652F20E02011717ABAC03D01791ABB0EC
:101E60001781ABB41785ABB21787AE50DF6EDF506A
:0E1E7000E552E552E5CFDAFFE7CFD9FF1200C9
:021E7E00D9CFBA
:101E8000E6FFDACFE6FFE1CFD9FFE2CFDAFFE65295
:101E9000E652D650DF6E010ED7CFDBFFDECF14F057
:101EA000DDCF15F014C0F3FF15C0F4FFE552E55285
:0C1EB000E552E5CFDAFFE7CFD9FF1200C2
:041EBC00D9CFE6FF95
:101EC000DACFE6FFE1CFD9FFE2CFDAFFFD0EDB503C
:101ED0007F0BD56ED76AD66AF294FD0EDBAE02D0C8
:101EE000F28A01D0F29AD58EE552E5CFDAFFE7CF3C
:041EF000D9FF120004
:0C1EF400D9CFE6FFDACFE6FFE1CFD9FF3F
:101F0000E2CFDAFFACAC04D0AC90020117B3AC80E6
:101F1000FD0EDB50AD6EE552E5CFDAFFE7CFD9FF1E
:021F20001200AD
:0E1F2200F36AF46AFF0EE124E96EFF0EE2207E
:101F3000EA6EED6607D02F0EEF6404D03A0EEF6024
:061F400001D0F32A12009B
:0A1F4600000EF36E00EE00F0080E2E
:101F500001D81200EA6002D0EE6AFCD7F350E960C3
:061F60001200EE6AFCD73E
:0A1F660012EE40F022EE40F0F86A9F
:101F7000019C1BEC0DF0E4EC0FF08DEC0CF0FBD7AA
:021F800012004D
:0E1F8200FF0EE350ACBA04D0AF6AAB8EAC8A4F
:0E1F9000949CACA2FED7AD6EF36EF46A120004
:021F9E00F36AE4
:101FA000F46AF32A0F0B05E0D890F336F436E80410
:041FB000FBE112003F
:0C1FB40030313233343536373839616251
:051FC00063646566008A
:021FC600120007
:021FC800120005
:021FCA00FEFF18
:041FCC000000000011
:071FD000000D0000010101FA
:00000001FF
